 nullws

 Timestamp is 4be8cf15 (Tue May 11 12:29:25 2010)

 Preferred load address is 10000000

 Start         Length     Name                   Class
 0001:00000000 00000004H .CRT$XCA                CODE
 0001:00000004 00000004H .CRT$XCZ                CODE
 0001:00000008 00000004H .CRT$XIA                CODE
 0001:0000000c 00000004H .CRT$XIZ                CODE
 0001:00000010 00000004H .CRT$XPA                CODE
 0001:00000014 00000004H .CRT$XPZ                CODE
 0001:00000018 00000004H .CRT$XTA                CODE
 0001:0000001c 00000004H .CRT$XTZ                CODE
 0001:00000020 000003d8H .rdata                  CODE
 0001:000003f8 00000023H .rdata$debug            CODE
 0001:0000041c 0000309cH .text                   CODE
 0001:000034b8 0000001cH .xdata                  CODE
 0001:000034d4 00000028H .idata$2                CODE
 0001:000034fc 00000014H .idata$3                CODE
 0001:00003510 00000138H .idata$4                CODE
 0001:00003648 000001eaH .idata$6                CODE
 0001:00003840 0000005bH .edata                  CODE
 0002:00000000 00000138H .idata$5                DATA
 0002:00000138 00000068H .data                   DATA
 0002:000001a0 00000050H .bss                    DATA
 0003:00000000 00000180H .pdata                  DATA

  Address         Publics by Value              Rva+Base       Lib:Object

 0000:00000000       ___safe_se_handler_table   00000000     <absolute>
 0000:00000000       ___safe_se_handler_count   00000000     <absolute>
 0001:00000000       __xc_a                     10001000     corelib0:crt0init.obj
 0001:00000004       __xc_z                     10001004     corelib0:crt0init.obj
 0001:00000008       __xi_a                     10001008     corelib0:crt0init.obj
 0001:0000000c       __xi_z                     1000100c     corelib0:crt0init.obj
 0001:00000010       __xp_a                     10001010     corelib0:crt0init.obj
 0001:00000014       __xp_z                     10001014     corelib0:crt0init.obj
 0001:00000018       __xt_a                     10001018     corelib0:crt0init.obj
 0001:0000001c       __xt_z                     1000101c     corelib0:crt0init.obj
 0001:00000098       ??_C@_0DI@GEDGMGKG@AddToClipRectList?3?5can?8t?5realloc@ 10001098     wince_ws.obj
 0001:000000d0       ??_C@_1BI@FPJLJJJA@?$AAD?$AAu?$AAm?$AAm?$AAy?$AAW?$AAi?$AAn?$AAd?$AAo?$AAw?$AA?$AA@ 100010d0     wince_ws.obj
 0001:000000e8       ??_C@_1EA@JHONGKOO@?$AAP?$AAV?$AAR?$AA2?$AAD?$AAQ?$AAu?$AAe?$AAr?$AAy?$AAB?$AAl?$AAi?$AAt?$AAs?$AAC?$AAo?$AAm?$AAp?$AAl?$AAe?$AAt?$AAe?$AA?5?$AAf?$AAa?$AAi?$AAl?$AAe?$AAd?$AA?4?$AA?$AA@ 100010e8     wince_ws.obj
 0001:00000128       ??_C@_0CK@PCGEFLPJ@WSEGL_CreateWindowDrawable?3?5Bad?5@ 10001128     wince_ws.obj
 0001:00000468       RegionsIdentical           10001468 f   wince_ws.obj
 0001:00000bf8       DummyWndProc               10001bf8 f   wince_ws.obj
 0001:00000c64       ForceDesktopRedraw         10001c64 f   wince_ws.obj
 0001:000013e8       WSEGL_GetFunctionTablePointer 100023e8 f   wince_ws.obj
 0001:00001c78       PVR2DEnumerateDevices      10002c78 f   libpvr2d:pvr2dinit.obj
 0001:00002048       PVR2DCreateDeviceContext   10003048 f   libpvr2d:pvr2dinit.obj
 0001:00002270       PVR2DDestroyDeviceContext  10003270 f   libpvr2d:pvr2dinit.obj
 0001:00002374       PVR2DGetFrameBuffer        10003374 f   libpvr2d:pvr2dmode.obj
 0001:000023b0       PVR2DGetDeviceInfo         100033b0 f   libpvr2d:pvr2dmode.obj
 0001:00002470       PVR2DMemAlloc              10003470 f   libpvr2d:pvr2dmem.obj
 0001:0000252c       PVR2DMemFree               1000352c f   libpvr2d:pvr2dmem.obj
 0001:000025f0       PVR2DQueryBlitsComplete    100035f0 f   libpvr2d:pvr2dblt.obj
 0001:000026cc       PVR2DSetPresentBltProperties 100036cc f   libpvr2d:pvr2dblt.obj
 0001:00002968       PVR2DPresentBlt            10003968 f   libpvr2d:pvr2dblt.obj
 0001:000029c4       DestroyFlipChain           100039c4 f   libpvr2d:pvr2dflip.obj
 0001:00002a94       PVR2DPresentFlip           10003a94 f   libpvr2d:pvr2dflip.obj
 0001:00002b34       PVR2DSetPresentFlipProperties 10003b34 f   libpvr2d:pvr2dflip.obj
 0001:00002c4c       ClientToScreen             10003c4c f   coredll:COREDLL.dll
 0001:00002c5c       GetClientRect              10003c5c f   coredll:COREDLL.dll
 0001:00002c6c       GetCurrentPositionEx       10003c6c f   coredll:COREDLL.dll
 0001:00002c7c       GetDC                      10003c7c f   coredll:COREDLL.dll
 0001:00002c8c       EndPaint                   10003c8c f   coredll:COREDLL.dll
 0001:00002c9c       BeginPaint                 10003c9c f   coredll:COREDLL.dll
 0001:00002cac       DefWindowProcW             10003cac f   coredll:COREDLL.dll
 0001:00002cbc       UnregisterClassW           10003cbc f   coredll:COREDLL.dll
 0001:00002ccc       DestroyWindow              10003ccc f   coredll:COREDLL.dll
 0001:00002cdc       UpdateWindow               10003cdc f   coredll:COREDLL.dll
 0001:00002cec       ShowWindow                 10003cec f   coredll:COREDLL.dll
 0001:00002cfc       CreateWindowExW            10003cfc f   coredll:COREDLL.dll
 0001:00002d0c       GetSystemMetrics           10003d0c f   coredll:COREDLL.dll
 0001:00002d1c       RegisterClassW             10003d1c f   coredll:COREDLL.dll
 0001:00002d2c       GetModuleHandleW           10003d2c f   coredll:COREDLL.dll
 0001:00002d3c       OutputDebugStringW         10003d3c f   coredll:COREDLL.dll
 0001:00002d4c       DeleteObject               10003d4c f   coredll:COREDLL.dll
 0001:00002d5c       CreateRectRgn              10003d5c f   coredll:COREDLL.dll
 0001:00002d6c       GetWindowLongW             10003d6c f   coredll:COREDLL.dll
 0001:00002d7c       GetRegionData              10003d7c f   coredll:COREDLL.dll
 0001:00002d8c       GetWindowRect              10003d8c f   coredll:COREDLL.dll
 0001:00002d9c       GetWindowRgn               10003d9c f   coredll:COREDLL.dll
 0001:00002dac       GetWindow                  10003dac f   coredll:COREDLL.dll
 0001:00002dbc       IsWindowVisible            10003dbc f   coredll:COREDLL.dll
 0001:00002dcc       SetThreadPriority          10003dcc f   coredll:COREDLL.dll
 0001:00002ddc       GetThreadPriority          10003ddc f   coredll:COREDLL.dll
 0001:00002dec       DllMain                    10003dec f   corelib0:dllmain.obj
 0001:00002f08       _DllMainCRTStartup         10003f08 f   corelib0:pegdmain.obj
 0001:00002f38       __GSHandlerCheckCommon     10003f38 f   corelib0:gshandler.obj
 0001:00002f74       __GSHandlerCheck           10003f74 f   corelib0:gshandler.obj
 0001:00002f98       __security_init_cookie     10003f98 f   corelib0:seccinit.obj
 0001:00002ff4       __security_check_cookie    10003ff4 f   corelib0:armsecgs.obj
 0001:00003008       __gsfailure                10004008 f   corelib0:armsecgs.obj
 0001:00003114       _cexit                     10004114 f   corelib0:cexit.obj
 0001:00003130       _initterm                  10004130 f   corelib0:crt0dat.obj
 0001:00003164       _cinit                     10004164 f   corelib0:crt0dat.obj
 0001:00003198       malloc                     10004198 f   corelib1:COREDLL.dll
 0001:000031a8       memcpy                     100041a8 f   corelib1:COREDLL.dll
 0001:000031b8       free                       100041b8 f   corelib1:COREDLL.dll
 0001:000031c8       fprintf                    100041c8 f   corelib1:COREDLL.dll
 0001:000031d8       _getstdfilex               100041d8 f   corelib1:COREDLL.dll
 0001:000031e8       realloc                    100041e8 f   corelib1:COREDLL.dll
 0001:000031f8       calloc                     100041f8 f   corelib1:COREDLL.dll
 0001:00003208       _XcptFilter                10004208 f   corelib1:COREDLL.dll
 0001:00003218       __C_specific_handler       10004218 f   corelib1:COREDLL.dll
 0001:00003228       __security_gen_cookie2     10004228 f   corelib1:COREDLL.dll
 0001:00003238       __report_gsfailure         10004238 f   corelib1:COREDLL.dll
 0001:00003248       PVRSRVDisconnect           10004248 f   srvclum:SRVCLUM.dll
 0001:00003258       PVRSRVCloseDCDevice        10004258 f   srvclum:SRVCLUM.dll
 0001:00003268       PVRSRVMemCopy              10004268 f   srvclum:SRVCLUM.dll
 0001:00003278       PVRSRVGetDCInfo            10004278 f   srvclum:SRVCLUM.dll
 0001:00003288       PVRSRVOpenDCDevice         10004288 f   srvclum:SRVCLUM.dll
 0001:00003298       PVRSRVFreeUserModeMem      10004298 f   srvclum:SRVCLUM.dll
 0001:000032a8       PVRSRVCallocUserModeMem    100042a8 f   srvclum:SRVCLUM.dll
 0001:000032b8       PVRSRVAcquireDeviceData    100042b8 f   srvclum:SRVCLUM.dll
 0001:000032c8       PVRSRVEnumerateDevices     100042c8 f   srvclum:SRVCLUM.dll
 0001:000032d8       PVRSRVEnumerateDeviceClass 100042d8 f   srvclum:SRVCLUM.dll
 0001:000032e8       PVRSRVConnect              100042e8 f   srvclum:SRVCLUM.dll
 0001:000032f8       PVRSRVUnmapDeviceClassMemory 100042f8 f   srvclum:SRVCLUM.dll
 0001:00003308       PVRSRVMapDeviceClassMemory 10004308 f   srvclum:SRVCLUM.dll
 0001:00003318       PVRSRVGetDCSystemBuffer    10004318 f   srvclum:SRVCLUM.dll
 0001:00003328       PVRSRVEnumDCDims           10004328 f   srvclum:SRVCLUM.dll
 0001:00003338       PVRSRVAllocUserModeMem     10004338 f   srvclum:SRVCLUM.dll
 0001:00003348       PVRSRVEnumDCFormats        10004348 f   srvclum:SRVCLUM.dll
 0001:00003358       PVRSRVDestroyDeviceMemContext 10004358 f   srvclum:SRVCLUM.dll
 0001:00003368       PVRSRVReleaseMiscInfo      10004368 f   srvclum:SRVCLUM.dll
 0001:00003378       SGXDestroyTransferContext  10004378 f   srvclum:SRVCLUM.dll
 0001:00003388       SGXCreateTransferContext   10004388 f   srvclum:SRVCLUM.dll
 0001:00003398       PVRSRVCreateDeviceMemContext 10004398 f   srvclum:SRVCLUM.dll
 0001:000033a8       PVRSRVGetMiscInfo          100043a8 f   srvclum:SRVCLUM.dll
 0001:000033b8       PVRSRVAllocDeviceMem       100043b8 f   srvclum:SRVCLUM.dll
 0001:000033c8       PVRSRVMemSet               100043c8 f   srvclum:SRVCLUM.dll
 0001:000033d8       PVRSRVFreeDeviceMem        100043d8 f   srvclum:SRVCLUM.dll
 0001:000033e8       PVRSRVUnwrapExtMemory      100043e8 f   srvclum:SRVCLUM.dll
 0001:000033f8       PVRSRVUnmapDeviceMemory    100043f8 f   srvclum:SRVCLUM.dll
 0001:00003408       PVRSRVEventObjectWait      10004408 f   srvclum:SRVCLUM.dll
 0001:00003418       SGX2DQueryBlitsComplete    10004418 f   srvclum:SRVCLUM.dll
 0001:00003428       PVRSRVClockus              10004428 f   srvclum:SRVCLUM.dll
 0001:00003438       PVRSRVReallocUserModeMem   10004438 f   srvclum:SRVCLUM.dll
 0001:00003448       SGXQueueTransfer           10004448 f   srvclum:SRVCLUM.dll
 0001:00003458       PVRSRVDestroyDCSwapChain   10004458 f   srvclum:SRVCLUM.dll
 0001:00003468       PVRSRVSwapToDCSystem       10004468 f   srvclum:SRVCLUM.dll
 0001:00003478       PVRSRVSwapToDCBuffer       10004478 f   srvclum:SRVCLUM.dll
 0001:00003488       PVRSRVSetDCDstRect         10004488 f   srvclum:SRVCLUM.dll
 0001:00003498       DisableThreadLibraryCalls  10004498 f   coredll:COREDLL.dll
 0001:000034a8       TerminateProcess           100044a8 f   coredll:COREDLL.dll
 0001:000034d4       __IMPORT_DESCRIPTOR_COREDLL 100044d4     coredll:COREDLL.dll
 0001:000034e8       __IMPORT_DESCRIPTOR_SRVCLUM 100044e8     srvclum:SRVCLUM.dll
 0001:000034fc       __NULL_IMPORT_DESCRIPTOR   100044fc     coredll:COREDLL.dll
 0002:00000000       __imp_ClientToScreen       10005000     coredll:COREDLL.dll
 0002:00000004       __imp_GetClientRect        10005004     coredll:COREDLL.dll
 0002:00000008       __imp_GetCurrentPositionEx 10005008     coredll:COREDLL.dll
 0002:0000000c       __imp_GetDC                1000500c     coredll:COREDLL.dll
 0002:00000010       __imp_EndPaint             10005010     coredll:COREDLL.dll
 0002:00000014       __imp_BeginPaint           10005014     coredll:COREDLL.dll
 0002:00000018       __imp_DefWindowProcW       10005018     coredll:COREDLL.dll
 0002:0000001c       __imp_UnregisterClassW     1000501c     coredll:COREDLL.dll
 0002:00000020       __imp_DestroyWindow        10005020     coredll:COREDLL.dll
 0002:00000024       __imp_UpdateWindow         10005024     coredll:COREDLL.dll
 0002:00000028       __imp_ShowWindow           10005028     coredll:COREDLL.dll
 0002:0000002c       __imp_CreateWindowExW      1000502c     coredll:COREDLL.dll
 0002:00000030       __imp_GetSystemMetrics     10005030     coredll:COREDLL.dll
 0002:00000034       __imp_RegisterClassW       10005034     coredll:COREDLL.dll
 0002:00000038       __imp_GetModuleHandleW     10005038     coredll:COREDLL.dll
 0002:0000003c       __imp_OutputDebugStringW   1000503c     coredll:COREDLL.dll
 0002:00000040       __imp_DeleteObject         10005040     coredll:COREDLL.dll
 0002:00000044       __imp_CreateRectRgn        10005044     coredll:COREDLL.dll
 0002:00000048       __imp_GetWindowLongW       10005048     coredll:COREDLL.dll
 0002:0000004c       __imp_GetRegionData        1000504c     coredll:COREDLL.dll
 0002:00000050       __imp_GetWindowRect        10005050     coredll:COREDLL.dll
 0002:00000054       __imp_GetWindowRgn         10005054     coredll:COREDLL.dll
 0002:00000058       __imp_GetWindow            10005058     coredll:COREDLL.dll
 0002:0000005c       __imp_IsWindowVisible      1000505c     coredll:COREDLL.dll
 0002:00000060       __imp_SetThreadPriority    10005060     coredll:COREDLL.dll
 0002:00000064       __imp_GetThreadPriority    10005064     coredll:COREDLL.dll
 0002:00000068       __imp_malloc               10005068     corelib1:COREDLL.dll
 0002:0000006c       __imp_memcpy               1000506c     corelib1:COREDLL.dll
 0002:00000070       __imp_free                 10005070     corelib1:COREDLL.dll
 0002:00000074       __imp_fprintf              10005074     corelib1:COREDLL.dll
 0002:00000078       __imp__getstdfilex         10005078     corelib1:COREDLL.dll
 0002:0000007c       __imp_realloc              1000507c     corelib1:COREDLL.dll
 0002:00000080       __imp_calloc               10005080     corelib1:COREDLL.dll
 0002:00000084       __imp__XcptFilter          10005084     corelib1:COREDLL.dll
 0002:00000088       __imp___C_specific_handler 10005088     corelib1:COREDLL.dll
 0002:0000008c       __imp___security_gen_cookie2 1000508c     corelib1:COREDLL.dll
 0002:00000090       __imp___report_gsfailure   10005090     corelib1:COREDLL.dll
 0002:00000094       __imp_DisableThreadLibraryCalls 10005094     coredll:COREDLL.dll
 0002:00000098       __imp_TerminateProcess     10005098     coredll:COREDLL.dll
 0002:0000009c       \177COREDLL_NULL_THUNK_DATA 1000509c     coredll:COREDLL.dll
 0002:000000a0       __imp_PVRSRVCloseDCDevice  100050a0     srvclum:SRVCLUM.dll
 0002:000000a4       __imp_PVRSRVGetDCInfo      100050a4     srvclum:SRVCLUM.dll
 0002:000000a8       __imp_PVRSRVOpenDCDevice   100050a8     srvclum:SRVCLUM.dll
 0002:000000ac       __imp_PVRSRVFreeUserModeMem 100050ac     srvclum:SRVCLUM.dll
 0002:000000b0       __imp_PVRSRVCallocUserModeMem 100050b0     srvclum:SRVCLUM.dll
 0002:000000b4       __imp_PVRSRVAcquireDeviceData 100050b4     srvclum:SRVCLUM.dll
 0002:000000b8       __imp_PVRSRVEnumerateDevices 100050b8     srvclum:SRVCLUM.dll
 0002:000000bc       __imp_PVRSRVEnumerateDeviceClass 100050bc     srvclum:SRVCLUM.dll
 0002:000000c0       __imp_PVRSRVConnect        100050c0     srvclum:SRVCLUM.dll
 0002:000000c4       __imp_PVRSRVUnmapDeviceClassMemory 100050c4     srvclum:SRVCLUM.dll
 0002:000000c8       __imp_PVRSRVMapDeviceClassMemory 100050c8     srvclum:SRVCLUM.dll
 0002:000000cc       __imp_PVRSRVGetDCSystemBuffer 100050cc     srvclum:SRVCLUM.dll
 0002:000000d0       __imp_PVRSRVEnumDCDims     100050d0     srvclum:SRVCLUM.dll
 0002:000000d4       __imp_PVRSRVAllocUserModeMem 100050d4     srvclum:SRVCLUM.dll
 0002:000000d8       __imp_PVRSRVEnumDCFormats  100050d8     srvclum:SRVCLUM.dll
 0002:000000dc       __imp_PVRSRVDestroyDeviceMemContext 100050dc     srvclum:SRVCLUM.dll
 0002:000000e0       __imp_PVRSRVReleaseMiscInfo 100050e0     srvclum:SRVCLUM.dll
 0002:000000e4       __imp_SGXDestroyTransferContext 100050e4     srvclum:SRVCLUM.dll
 0002:000000e8       __imp_SGXCreateTransferContext 100050e8     srvclum:SRVCLUM.dll
 0002:000000ec       __imp_PVRSRVCreateDeviceMemContext 100050ec     srvclum:SRVCLUM.dll
 0002:000000f0       __imp_PVRSRVGetMiscInfo    100050f0     srvclum:SRVCLUM.dll
 0002:000000f4       __imp_PVRSRVAllocDeviceMem 100050f4     srvclum:SRVCLUM.dll
 0002:000000f8       __imp_PVRSRVMemSet         100050f8     srvclum:SRVCLUM.dll
 0002:000000fc       __imp_PVRSRVFreeDeviceMem  100050fc     srvclum:SRVCLUM.dll
 0002:00000100       __imp_PVRSRVUnwrapExtMemory 10005100     srvclum:SRVCLUM.dll
 0002:00000104       __imp_PVRSRVUnmapDeviceMemory 10005104     srvclum:SRVCLUM.dll
 0002:00000108       __imp_PVRSRVEventObjectWait 10005108     srvclum:SRVCLUM.dll
 0002:0000010c       __imp_SGX2DQueryBlitsComplete 1000510c     srvclum:SRVCLUM.dll
 0002:00000110       __imp_PVRSRVClockus        10005110     srvclum:SRVCLUM.dll
 0002:00000114       __imp_PVRSRVReallocUserModeMem 10005114     srvclum:SRVCLUM.dll
 0002:00000118       __imp_SGXQueueTransfer     10005118     srvclum:SRVCLUM.dll
 0002:0000011c       __imp_PVRSRVDestroyDCSwapChain 1000511c     srvclum:SRVCLUM.dll
 0002:00000120       __imp_PVRSRVSwapToDCSystem 10005120     srvclum:SRVCLUM.dll
 0002:00000124       __imp_PVRSRVSwapToDCBuffer 10005124     srvclum:SRVCLUM.dll
 0002:00000128       __imp_PVRSRVSetDCDstRect   10005128     srvclum:SRVCLUM.dll
 0002:0000012c       __imp_PVRSRVDisconnect     1000512c     srvclum:SRVCLUM.dll
 0002:00000130       __imp_PVRSRVMemCopy        10005130     srvclum:SRVCLUM.dll
 0002:00000134       \177SRVCLUM_NULL_THUNK_DATA 10005134     srvclum:SRVCLUM.dll
 0002:00000198       __security_cookie          10005198     corelib0:seccinit.obj
 0002:0000019c       __security_cookie_complement 1000519c     corelib0:seccinit.obj
 0002:000001e0       _exitflag                  100051e0     corelib0:cexit.obj
 0002:000001e4       __onexitend                100051e4     <common>
 0002:000001e8       __onexitbegin              100051e8     <common>
 0002:000001ec       _pRawDllMain               100051ec     <common>

 entry point at        0001:00002f08

 Static symbols

 0001:0000041c       FreeRegions                1000141c f   wince_ws.obj
 0001:00000524       AddToClipRectList          10001524 f   wince_ws.obj
 0001:000005b8       SubtractRects              100015b8 f   wince_ws.obj
 0001:00000970       WSEGLWCEGetWindowInfo      10001970 f   wince_ws.obj
 0001:00000a1c       WSEGL_IsDisplayValid       10001a1c f   wince_ws.obj
 0001:00000a54       WSEGL_InitialiseDisplay    10001a54 f   wince_ws.obj
 0001:00000d58       WSEGL_DeleteDrawable       10001d58 f   wince_ws.obj
 0001:00000e5c       WSEGL_CloseDisplay         10001e5c f   wince_ws.obj
 0001:00000e9c       WSEGL_CreateWindowDrawable 10001e9c f   wince_ws.obj
 0001:000011fc       WSEGL_CreatePixmapDrawable 100021fc f   wince_ws.obj
 0001:00001204       WSEGL_SwapControlInterval  10002204 f   wince_ws.obj
 0001:0000124c       WSEGL_WaitNative           1000224c f   wince_ws.obj
 0001:0000125c       WSEGL_CopyFromDrawable     1000225c f   wince_ws.obj
 0001:00001264       WSEGL_CopyFromPBuffer      10002264 f   wince_ws.obj
 0001:0000126c       WSEGL_GetDrawableParameters 1000226c f   wince_ws.obj
 0001:000013f4       WSEGLWCEGetClipRect        100023f4 f   wince_ws.obj
 0001:00001938       WSEGL_SwapDrawable         10002938 f   wince_ws.obj
 0001:00001e60       InitDisplayDevice          10002e60 f   libpvr2d:pvr2dinit.obj
 0001:000027b4       AltPresentBlt              100037b4 f   libpvr2d:pvr2dblt.obj
 0001:00002e0c       _DllMainCRTStartupHelper   10003e0c f   corelib0:pegdmain.obj
 0001:0000304c       doexit                     1000404c f   corelib0:cexit.obj
